:020000040000FA
:06000000020091022C87B2
:030023000229446B
:03002B00022C9B09
:10003B00022B5F53D9BF79012200000080FB120015
:10004B003EB9000302008BE49010007850790A80CF
:10005B0002F0A3D8FCD9FA90194FAA82AB83900077
:10006B00A0780D79028015E493A3AC82AD838A82CC
:10007B008B83F0A3AA82AB838C828D83D8E9D9E7DB
:10008B00122D1D12004475D0007581BF75100075BF
:10009B001110020049506C656173652070726573B5
:1000AB007320616E79206B657920746F20636F6E9E
:1000BB0074696E75652E2E2E203F007C205452499C
:1000CB0047207C203530306E732F64207C203235F6
:1000DB002E30562F64207C2032352E30562F642044
:1000EB007C3F007C2053796E63207C20496E74200A
:1000FB007C205A20434841207C205A2043484220F0
:10010B007C204143204143207C3F0032352E30562A
:10011B002F643F0041433F0044433F00496E743F0F
:10012B000053796E633F0072616E67653A0000029F
:10013B0059802054524947203F0000002035303071
:10014B006E732F64203F2032352E30562F64203FA4
:10015B002032352E30562F64203F2053796E63208A
:10016B003F00000020496E74203F00000000205A21
:10017B0020434841203F0000205A20434842203F63
:10018B00000020464654203F000000000000000005
:10019B0000000000000001E52FE6FF00F80140071A
:1001AB0007CAC0E0E6F0A308DAFAD0E0FA22C3E40B
:1001BB0098F8E499F91201FA8026C3E49AFAE49BC1
:1001CB00FBE920E7E91201FAE498F8E499F922C374
:1001DB00E498F8E499F91201FAE498F8E499F9C370
:1001EB00E49AFAE49BFB22EB20E7CFE920E7E0B9A6
:1001FB000010BB0008E88AF084F8AAF022E4FBC8E0
:10020B00FA22EB70227B10C833C8C933C9335007AD
:10021B00C39AC3DBF280069A50012ADBEAC833F497
:10022B00C8C933F4C9FA2275F008E4C833C8C93316
:10023B00C933C99AC99B5004C92AC93BD5F0ECFBF9
:10024B00C833F4C8E4C9FA22600D08C6A2E713C686
:10025B0018C613C6D5E0F322700422600D18C6C36E
:10026B0033C608C633C6D5E0F41822251010AF08E4
:10027B00F510400215118008F51040021511D2AF90
:10028B0022C0D0251010AF08F510500205118008C0
:10029B00F51050020511D2AFD0D0222510F58210E7
:1002AB00AF08F510400215118008F510400215112A
:1002BB00D2AF851183222510F582E43511F5832207
:1002CB002510C582C0E0E51134FFC583C0E0E51001
:1002DB00C3958224F9F8E4C5A8858311858210C5DE
:1002EB00A8E8CEF0A3E520F0A37808E608F0A3DE9B
:1002FB00FAEFF0A3E58124FBF8E608F0A3E608F09B
:10030B00A30808E608F0A3E608F0A315811581D031
:10031B00E0FED0E0F815811581E8C0E0EEC0E022E8
:10032B00851183851082E0A3FEE0A3F5207808E019
:10033B00A3F608DFFAE0A3FFE0A3C0E0E0A3C0E070
:10034B00E0A3C0E0E0A3C0E0E4C5A88582108583EC
:10035B0011C5A8D083D0822274028000C0E0F404BF
:10036B001202A6D0E01201AC22D083D082C5F0E4F9
:10037B0093A3C5F0C395F0F5F0E493A3C395F040B8
:10038B0005E5F0048001E475F002A42582F582E511
:10039B00F03583F583E493A3C0E0E493C0E022D06F
:1003AB0083D082E9C0E0E493A3C386F0C5F095F057
:1003BB00F908E493A386F0C5F095F0700BE493A3D2
:1003CB00C3994005E9048002A3E475F002A42582D9
:1003DB00F582E5F03583F583D0E0F9E493A3C0E033
:1003EB00E493C0E022D083D082CCC0E0E493A3603E
:1003FB000612041A1470FAE493A36006120439145B
:10040B0070FAD0E0FCE493A3C0E0E493C0E022C018
:10041B00E0E493A3D39C5010E493A3C39C400AD075
:10042B00E0D0E0D0E002040DA3A3A3D0E022C0E013
:10043B00E493A36C7009D0E0D0E0D0E002040DA3EC
:10044B00A3D0E022008040C020A060E0109050D0EC
:10045B0030B070F0088848C828A868E8189858D8B1
:10046B0038B878F8048444C424A464E4149454D4B1
:10047B0034B474F40C8C4CCC2CAC6CEC1C9C5CDC51
:10048B003CBC7CFC028242C222A262E2129252D299
:10049B0032B272F20A8A4ACA2AAA6AEA1A9A5ADA51
:1004AB003ABA7AFA068646C626A666E6169656D651
:1004BB0036B676F60E8E4ECE2EAE6EEE1E9E5EDEF1
:1004CB003EBE7EFE018141C121A161E1119151D15D
:1004DB0031B171F1098949C929A969E9199959D921
:1004EB0039B979F9058545C525A565E5159555D521
:1004FB0035B575F50D8D4DCD2DAD6DED1D9D5DDDC1
:10050B003DBD7DFD038343C323A363E3139353D308
:10051B0033B373F30B8B4BCB2BAB6BEB1B9B5BDBC0
:10052B003BBB7BFB078747C727A767E7179757D7C0
:10053B0037B777F70F8F4FCF2FAF6FEF1F9F5FDF60
:10054B003FBF7FFF00402060105030700848286884
:10055B001858387804442464145434740C4C2C6CA0
:10056B001C5C3C7C02422262125232720A4A2A6A98
:10057B001A5A3A7A06462666165636760E4E2E6E60
:10058B001E5E3E7E0141216111513171094929697C
:10059B001959397905452565155535750D4D2D6D50
:1005AB001D5D3D7D03432363135333730B4B2B6B48
:1005BB001B5B3B7B07472767175737770F4F2F6F10
:1005CB001F5F3F7F00402060105030700848286844
:1005DB001858387804442464145434740C4C2C6C20
:1005EB001C5C3C7C02422262125232720A4A2A6A18
:1005FB001A5A3A7A06462666165636760E4E2E6EE0
:10060B001E5E3E7E014121611151317109492969FB
:10061B001959397905452565155535750D4D2D6DCF
:10062B001D5D3D7D03432363135333730B4B2B6BC7
:10063B001B5B3B7B07472767175737770F4F2F6F8F
:10064B001F5F3F7F00000000000000000000000063
:10065B00000000000000000000100000000000007F
:10066B00001E000000000000001FC0000000000082
:10067B00001FF80000000000000FFF00000000004A
:10068B000001FFE00000000000003FFC0000000044
:10069B00000007FC00000000000000FC0000000050
:1006AB00000000FC00000000000003F80000000048
:1006BB00000007E0000018E801000FC0000018EC74
:1006CB0000001F800000181E00007E000000180EA6
:1006DB008000FC0000001803C001F80000001801A6
:1006EB00E107F00000001800790FC00000001800AF
:1006FB003E1F8000000018000E1FC00000001800F5
:10070B00031FF800000018000F0FFF000000180077
:10071B000D01FFE00000180079003FFC00001800FD
:10072B00F00007FC00001801C00000FC00001803DB
:10073B008000001C00001807018000000000181C3E
:10074B00000000000000181800000000000008B0B6
:10075B0000100000000009F0001E0000000019C08E
:10076B00001FC00000001F01199FF80000001E9918
:10077B00001FFF000098DC000019FFE00880380024
:10078B0000183FE008007800011837E00001D8009E
:10079B00011830E00001880000183060000B1800D1
:1007AB0000183060000E080000183060001C1800A4
:1007BB0000183060007808000198306000E01800E5
:1007CB000018306001C008000018006007800800A6
:1007DB00001800600F0018000008006012000800ED
:1007EB00000000601C001800018000607800080009
:1007FB00000000607000180000000060600008003E
:10080B00001000003C000800001E00001F00080044
:10081B00009FC00007800800019FF80001E8080056
:10082B00000FFF00007808000001FFE0002E080019
:10083B0000003FE0000B8800008007E00001C808C3
:10084B00898000E000017C88880000000000FC88A3
:10085B000000000000489E000010000008801F40B0
:10086B00001E0000000009D0019FC000000008F42A
:10087B00001FF80000000C2C001FFF000000080FE9
:10088B008019FFE00000080580183FE000000C0015
:10089B00C01807E000000800F99800E000000C0009
:1008AB003C180000000008000F18000000000C00AE
:1008BB0007180000000008000318000000000C00DF
:1008CB000698000000000C001C98000000000800B7
:1008DB003818000000000C00680800000000080039
:1008EB00E000000000000C038080000000000807FF
:1008FB000080000000000C1C000000000000081825
:10090B000000000000000838000E000000000CE0A2
:10091B00001F0000400008C0009F800000000F84F3
:10092B00881F800000000EC8001D8F00000C5C00AB
:10093B00001C1FE044845C00001C1FF804C07C00FA
:10094B00001C1FF800006C00009C1CFC0001AC009C
:10095B00001C1C1C00038C00001C1C1C00070C0042
:10096B00001C1C1C401C0800001C1C1C0018040054
:10097B00009C1C1C00680400009C1C1C00E00C006C
:10098B00001C1C1C01800C00001C1C1C03800C0098
:10099B00001E1C1C46000400009FDC1C1A000C00EF
:1009AB00008FFC1C180004000007FC1C380004001E
:1009BB000001FC7C70000C000000387C7B00040004
:1009CB000000007C4F000C000080007C05A00400A0
:1009DB000000000000E80C0000000000003E0400D6
:1009EB0000000000000F0C00000000004003A400FA
:1009FB001F9E00000002E42AFF9FC00000007C7FC6
:100A0B00C01FF8000000FFC0001FFF0000BFAE803A
:100A1B000019FFC07FD00DC000983FE0200005B843
:100A2B00001807E00000041A001800E00000040E94
:100A3B000018006000000407C018006000000401EB
:100A4B00C0180060400004007898006000000400AB
:100A5B001C18006000000400071800600000040070
:100A6B00079E006000000400019F806040000400AE
:100A7B00038F8860400004000E878F600000040025
:100A8B00080107E000000400380007E00000040044
:100A9B00F00003E000000402800000C040000401ED
:100AAB008000000000000406000000000000041697
:100ABB00001E00000000041C001FC00000000448C2
:100ACB00001FF800000004E0001FFF00400004C0FE
:100ADB004419FFC00000078400183FE000002E00FF
:100AEB00001807E000040C00001800E000041C00D4
:100AFB000018006044003400001800600000500033
:100B0B00001800600000E40000180060000384007F
:100B1B00001800600005040000180060400C040081
:100B2B000018006000180400001800600078040032
:100B3B00001E006000400400001FC06001C00400E4
:100B4B00000FF860038000000007FF604500040001
:100B5B000001FFE00C00000000003FE01800040063
:100B6B00000007E010000400000000C018000200A5
:100B7B00000000003E0004000000000005A004007F
:100B8B000000000000D00000001000000011040065
:100B9B00001E0000000E0000001FC0000005C0007A
:100BAB00001FF8000001E400000FFF0000003400FC
:100BBB000001FFE000001E4000007FE000004780C6
:100BCB00000067E0002004E0000060E0400000ACA3
:100BDB00000060600000000E000060600000040375
:100BEB002000606000000401200060600000040130
:100BFB0060006060000000003C00606000000000CE
:100C0B000E00606000000000030060600000040044
:100C1B00018078600000000001807FE00000000090
:100C2B0002003FE00000040006001FE0000000008F
:100C3B000C0007E000000400180000C000000400D6
:100C4B006010000000000400A01E00000000040162
:100C5B00801FC00000000407801FF8000000000484
:100C6B00001FFF000000000C0019FFE0000004381B
:100C7B0000183FE0000004A0001837E0000000E07F
:100C8B00001830E0000003800018306000000700FF
:100C9B0000183060000006000018306000000C00E7
:100CAB0000183060000018000018306000001400BD
:100CBB00001830600000E0000018006000018400A4
:100CCB00001800600004000000080060000604002B
:100CDB000000006000120400000000600010000023
:100CEB0000000060002004000000006000600000B5
:100CFB000000000000C000000000000001800400A4
:100D0B000000000002000000000000000C000000CA
:100D1B000000000008000400000000000C000400AC
:100D2B0000000000058004000000000001400400EA
:100D3B00000000000030000000000000001D040057
:100D4B0000000000000D4000000000000000D0007B
:100D5B00000000000000B0000000000000001400C4
:100D6B000000000000000000000000000000000078
:100D7B000010000000000000001C0000000000003C
:100D8B00001E000000000000001F0000000000001B
:100D9B00001F000000000000001F81000000000089
:100DAB00001F81E000000000001DC1F800000000E2
:100DBB00001DC1F800000000001CE0FC003FF01F0C
:100DCB00F81CE01C003FF01FF81C701C0003000116
:100DDB00981C701C00030001981C381C00030001B8
:100DEB00981C381C00030001981C1C1C00030001FC
:100DFB00981C1C1C00030000181E0E1C0003000096
:100E0B00181FC61C00030000180FC71C003FF00082
:100E1B000007C3FC003FF000000183FC0000000052
:100E2B00080001FC00000000780000FC000000013D
:100E3B00F00000080000000F800000000000101EF2
:100E4B00000000000000F01E000000000003E0079F
:100E5B0080000000001F0000F0100000003C0000AC
:100E6B00381E0000003C0000F81E0000000F0003BD
:100E7B00C01E00000001E01E001E00000000701CE0
:100E8B00000E00000001F00F0000000000078001C1
:100E9B00E0000000003C000078000000003800007B
:100EAB0008000000001E0000000000000003C0004E
:100EBB00000000000000F000000000000000100027
:100ECB000000000000000000000000000000000017
:100EDB00000E000000000000001FC000000000001A
:100EEB00001FF80000000000001FFF0000000000C2
:100EFB00001DFFE000000000041C3FF80000000094
:100F0B00041C07F800000000061C00FC0000001F7A
:100F1B00FE1C001C0000001FFE1C001C000000003B
:100F2B00001C001C001C3800001C001C003C3C007A
:100F3B00001C001C00300C00001C001C00300C00BE
:100F4B00001C001C00300C00001C001C00318C002D
:100F5B00001C001C00318C00001E001C00318C009A
:100F6B00001FC01C00318C00000FF81C00318C00DE
:100F7B000007FF1C003FFC000001FFFC001F780076
:100F8B0000003FFC00000000000007FC0000000018
:100F9B00000000FC0000001C000000000000001C12
:100FAB00000000000000001C00000000000000001A
:100FBB0000000000003800000000000000380000B6
:100FCB0000000000003800000000000000000000DE
:100FDB000000000000000000000000000000000EF8
:100FEB001C0000000000001E1E0000000000001886
:100FFB000600000000000018060000000019F018A1
:10100B00060000000030FC18C60000000030CC18B1
:10101B00C60000000030CC18C60000000030CC1811
:10102B00C60000000030CC18C60000000030CC1FFA
:10103B00FE0000000030CC0FBC0000000030CC00E4
:10104B00000000000030CC000000000000198C00F4
:10105B0000000000001F800000000000000F0000D7
:10106B000000000000000000000000000000001F56
:10107B00FE0000000000001FFE0000000000001832
:10108B000600000000000018060000000000001819
:10109B000600000000000018060000000000001809
:1010AB0006000000000000180600000000000018F9
:1010BB000600000000000018060000000000001CE5
:1010CB000E0000000000000E1C00000000000007D6
:1010DB00F800000000000003F0000000000000001A
:1010EB0000000000000000000000000000000000F5
:1010FB0000000000000000000000000000000000E5
:10110B0000000000000000000000FF33FF33000070
:10111B0000000000000007000700000000000700AF
:10112B00070000002001FE1FFE1F20012001FE1FF3
:10113B00FE1F200138063C0E6408FF3FFF3F840969
:10114B001C0F18071E30331C1E07C00170001C1E1D
:10115B000733011E1E1FB331E120E120B3311E1FE7
:10116B00001B80310000000000000B000700000096
:10117B000000000000000000F807FF3F07380000E8
:10118B000000000000000000000000000000000054
:10119B000000000000000000000000000000000044
:1011AB000000000000000000000000000000000034
:1011BB000000000000000000000000000000000024
:1011CB000000000000000000000000000000000014
:1011DB0000000000000000000000003000300000A4
:1011EB00000000000030003C000FC003F0003C008A
:1011FB000F000300FC0FFE1F0336812161201B3003
:10120B00FE1FFC0F042004200620FF3FFF3F0020A1
:10121B00002000200C380E3C032601238121C32023
:10122B007E203C20061803304120412041204120E4
:10123B00E330BE1F000FE00FFC081F08833F803F09
:10124B00000800083F0C3F1C213021202120613079
:10125B00C11F810FE00FF81F5C3046204320C130C7
:10126B00811F010F010001000100013C813FF103CF
:10127B007F000F001C0FBE1FE33041204120E330E5
:10128B00BE1F1C0F3C207E20C32081308118830E93
:10129B00FE07FC0100000000000000000000000041
:1012AB000000000000000000000000000000000033
:1012BB000000000000000000000000000000000023
:1012CB00000000002001200120012001200120014D
:1012DB0020012001000000000000000000000000C1
:1012EB0000000000000000000000000000000000F3
:1012FB0000000000000000000000000000000000E3
:10130B0000000000FC3FFE3F03010101010103014E
:10131B00FE3FFC3FFF3FFF3F412041204120E33098
:10132B00BE1F1C0FFC0FFE1F0330012001200330DA
:10133B000E1C0C0CFF3FFF3F012001200120073842
:10134B00FE1FF807FF3FFF3F412041204120412076
:10135B0041200120FF3FFF3F810081008100810080
:10136B0081000100FC0FFE1F033001208120833020
:10137B008E1F8C0FFF3FFF3F40004000400040009E
:10138B00FF3FFF3F012001200120FF3FFF3F0120D6
:10139B0001200120000C001C003000200020003038
:1013AB00FF1FFF0FFF3FFF3FC000E00138071C0E80
:1013BB000F3C0330FF3FFF3F0020002000200020A8
:1013CB0000200020FF3FFF3F7800C003C0037800E0
:1013DB00FF3FFF3FFF3FFF3F1C007000C0010007B6
:1013EB00FF3FFF3F00000000000000000000000076
:1013FB0000000000FF3FFF3F810081008100C30020
:10140B007E003C0000000000000000000000000017
:10141B0000000000FF3FFF3F810081008101C31FDF
:10142B007E3E3C203C0C7E1C6330E120C12183318D
:10143B008E1F0C0F030003000300FF3FFF3F030051
:10144B0003000300FF0FFF1F0030002000200030BF
:10145B00FF1FFF0F3F00FF01C00F003C003CC00F00
:10146B00FF013F00FF01FF3F003EC001C001003EF6
:10147B00FF3FFF0100000000000000000000000023
:10148B000000000000000000000000000000000051
:10149B00000000000138013E8127C1216120392065
:1014AB001F200720000000000000000000000000CB
:1014BB000000000000000000000000000000000021
:1014CB000000000000000000000000000000000011
:1014DB000000000000000000000000000000000001
:1014EB0000000000000000000000000000000000F1
:1014FB0000000000000000000000000000000000E1
:10150B0000000000001E403F20212021202120113F
:10151B00E03FC03FFF3FFF3F4010202020206030C6
:10152B00C01F800F800FC01F603020202020202084
:10153B0060304010800FC01F6030202020204010F2
:10154B00FF3FFF3F800FC01F60322022202260220E
:10155B00C033801320002000FE3FFF3F21002100FD
:10156B00230002008007C00F6018201020104008D5
:10157B00E03FE03F00000000000000000000000022
:10158B0000000000000020202020E33FE33F00206C
:10159B000020000000000000000000000000000020
:1015AB0000000000FC3FFC3F00060007800DC01848
:1015BB0060302020000001200120FF3FFF3F002072
:1015CB0000200000E03FE03F6000C01FC01F600034
:1015DB00E03FC03FE03FE03F4000200020006000C4
:1015EB00C03F803F800FC01F603020202020603024
:1015FB00C01F800FE03FE03F400420082008600C34
:10160B00C007800300000000000000000000000085
:10161B0000000000E03FE03FC000400060006000C1
:10162B0060004000C010E031202120232026202420
:10163B00603C4018000020002000FE1FFE3F2020D1
:10164B0020200000E01FE03F0020002000200010C1
:10165B00E03FE03FF003F007001C00300030001CBF
:10166B00F007F00300000000000000000000000085
:10167B00000000000000000000000000000000005F
:10168B0000000000E001E027002600380018000EE3
:10169B00E007E00120302038202C20262023A02139
:1016AB00E0206020000000000000000000000000AF
:1016BB0000000000000000000000FF3FFF3F0000A3
:1016CB00000000000000000000000000000000000F
:1016DB0000000000000000000000000000000000FF
:1016EB0000000000000000000000000000000000EF
:1016FB0000000000000000000000000000000000DF
:10170B0000000000000000000000000000000000CE
:10171B0000000000000102030405060708090A0B7C
:10172B000C0D0E0F101112131415161718191A1B76
:10173B001C1D1E1F202122232425262728292A2B66
:10174B002C2D2E2F303132333435363738393A3B56
:10175B003C3D3E3F404142434445464748494A4B46
:10176B004C4D4E4F505152535455565758595A5B36
:10177B005C5D5E5F000000000000000000000000E8
:10178B00000000000000000000000000000000004E
:10179B00000000000000000000000000000000003E
:1017AB00000000000000000000000000000000002E
:1017BB00000000000000000000000000000000001E
:1017CB00000000000000000000000000000000000E
:1017DB0000000000000000000000000000000000FE
:1017EB0000000000000000000000000000000000EE
:1017FB00000000000C000B000A00090008000A00A2
:10180B00090008003132356D3F3235306D3F3632CD
:10181B00356D3F312E32353F322E35303F362E323D
:10182B00353F31322E353F32352E303FFFFF000032
:10183B00020004000600080012001C0026004E00E7
:10184B00620076008A009E00B200C600EE00160110
:10185B002A013E0166018E0156021E03E6030200B9
:10186B00040008003530306E733F312E3075733FF6
:10187B00322E3075733F332E3075733F342E3075E7
:10188B00733F352E3075733F31302075733F3135D3
:10189B002075733F32302075733F34302075733FA2
:1018AB0035302075733F36302075733F37302075D8
:1018BB00733F38302075733F39302075733F3130AB
:1018CB003075733F31323075733F31343075733F40
:1018DB0031353075733F31363075733F3138307574
:1018EB00733F32303075733F33303075733F343064
:1018FB003075733F35303075733F312E306D733F1C
:10190B00322E306D733F342E306D733F3235306E67
:10191B00733F3530306E733F312E3075733F312E40
:10192B003575733F322E3075733F322E3575733FDD
:10193B0035202075733F372E3575733F3130207549
:10194B00733F32302075733F32352075733F333020
:10195B002075733F33352075733F34302075733FDB
:10196B0034352075733F35302075733F3630207515
:10197B00733F37302075733F37352075733F3830E1
:10198B002075733F39302075733F31303075733F9D
:10199B0031353075733F32303075733F32353075BA
:1019AB00733F35303075733F312E306D733F322EB0
:1019BB00306D733F75B9807A14001AEA70FB43B926
:1019CB00C0E5B9E5B9A2E550FA75A90275B2832253
:1019DB00C082C0831219BF75A40D75A5E775A70149
:1019EB0075D40F75D50775DF0175E10575E24243B7
:1019FB008805E58875E401D2A8C2AA759810758D83
:101A0B000D538EF4E58E438E08858D8B53890FE530
:101A1B0089438920D28E7401901A50F0D2ACD28CAB
:101A2B00438922E589438E0CE58E758CB075C18098
:101A3B0043E60175D80053D9BF75D90275DA4275E3
:101A4B00DB4275FC0775EA07D2DE75C80475CA015F
:101A5B0075CB01C2ADC283D282D280C292D291D257
:101A6B0090D2B0C296D296D2AF02293FD296D282F2
:101A7B00D29275A6FFD291C291D291D283C29275A6
:101A8B00A083C280D280D29275A002C280D280C2C3
:101A9B0083D283C29275A085C280D280D29275A068
:101AAB0003C280D280C283D283C29275A08CC280C3
:101ABB00D280D29275A093C280D280C283D283C2CD
:101ACB009275A091C280D280D29275A001C280D2B1
:101ADB0080C283D283C29275A083C280D280D292FD
:101AEB0075A000C280D280C283D283C29275A03E01
:101AFB00C280D280D29275A0B0C280D280C283D273
:101B0B0083C29275A03FC280D280D29275A003C2CD
:101B1B0080D280C283D283C29275A040C280D28011
:101B2B00D29275A010C280D280C283D283C292752A
:101B3B00A041C280D280D29275A056C280D280C200
:101B4B0083D283C29275A042C280D280D29275A0FA
:101B5B0013C280D280C283D283C29275A043C2804B
:101B6B00D280D29275A046C280D280C283D283C269
:101B7B009275A044C280D280D29275A023C280D22B
:101B8B0080C283D283C29275A045C280D280D2928A
:101B9B0075A076C280D280C283D283C29275A046D2
:101BAB00C280D280D29275A000C280D280C283D272
:101BBB0083C29275A047C280D280D29275A05EC2BA
:101BCB0080D280C283D283C29275A048C280D28059
:101BDB00D29275A04FC280D280C283D283C292753B
:101BEB00A049C280D280D29275A040C280D280C25E
:101BFB0083D283C29275A017C280D280D29275A075
:101C0B0061C280D280C283D283C29275A02BC28064
:101C1B00D280D29275A0F9C280D280C283D283C205
:101C2B009275A01BC280D280D29275A014C280D2B2
:101C3B0080C283D283C29275A01AC280D280D29204
:101C4B0075A011C280D280C283D283C29275A01CB0
:101C5B00C280D280D29275A00DC280D280C283D2B4
:101C6B0083C29275A01FC280D280D29275A03DC252
:101C7B0080D280C283D283C29275A019C280D280D7
:101C8B00D29275A00AC280D280C283D283C29275CF
:101C9B00A019C280D280D29275A01AC280D280C203
:101CAB0083D283C29275A019C280D280D29275A0C2
:101CBB0012C280D280C283D283C29275A01EC28010
:101CCB00D280D29275A020C280D280C283D283C22E
:101CDB009275A03CC280D280D29275A060C280D295
:101CEB0080C283D283C29275A03DC280D280D29231
:101CFB0075A040C280D280C283D283C29275A034B9
:101D0B00C280D280D29275A038C280D280C283D2D8
:101D1B0083C29275A035C280D280D29275A038C290
:101D2B0080D280C283D283C29275A024C280D2801B
:101D3B00D29275A038C280D280C283D283C29275F0
:101D4B00A024C280D280D29275A03CC280D280C225
:101D5B0083D283C29275A016C280D280D29275A014
:101D6B001CC280D280C283D283C29275A001C28072
:101D7B00D280D29275A006C280D280C283D283C297
:101D8B009275A055C280D280D29275A000C280D22B
:101D9B0080C283D283C29275A002C280D280D292BB
:101DAB0075A000C280D280C283D283C29275A00379
:101DBB00C280D280D29275A000C280D280C283D260
:101DCB0083C29275A004C280D280D29275A000C249
:101DDB0080D280C283D283C29275A005C280D2808A
:101DEB00D29275A0EFC280D280C283D283C2927589
:101DFB00A006C280D280D29275A000C280D280C2CF
:101E0B0083D283C29275A007C280D280D29275A072
:101E1B0000C280D280C283D283C29275A008C280D6
:101E2B00D280D29275A001C280D280C283D283C2EB
:101E3B009275A009C280D280D29275A08FC280D237
:101E4B0080C283D283C29275A022C280D280D292EA
:101E5B00C28375A60075A0FF2275A6FFD283C2921E
:101E6B0075A003C280D280D29289A0C280D280C2D8
:101E7B0083D283C29275A006C280D280D292EBF538
:101E8B00A0C280D280C283D283C29275A007C280C7
:101E9B00D280D292EAF5A0C280D280C283D283C212
:101EAB009275A022C280D280D292C2832274F81281
:101EBB0002CB74081202C1E0FEA3E0FFD283C292F0
:101ECB0075A002C280D280D29275A000C280D2804F
:101EDB00C283D283C29275A003C280D280D2928970
:101EEB00A0C280D280C283D283C29275A004C2806A
:101EFB00D280D29275A000C280D280C283D283C21C
:101F0B009275A005C280D280D2928CA0C280D28062
:101F1B00C283D283C29275A006C280D280D292EBCA
:101F2B00F5A0C280D280C283D283C29275A007C2B1
:101F3B0080D280D292EAF5A0C280D280C283D283B3
:101F4B00C29275A008C280D280D292EFF5A0C28057
:101F5B00D280C283D283C29275A009C280D280D2B2
:101F6B0092EEF5A0C280D280C283D283C29275A0BA
:101F7B0022C280D280D292C28302236974F71202EA
:101F8B00CB74091202C1E0F508A3E0F5097E987F36
:101F9B009E75A6FF7808120363121EB87402120214
:101FAB008CD283C29275A022C280D280D292C2837D
:101FBB00901047E0FAA3E0D283F5A0C280D280EA6A
:101FCB00F5A0C280D280C283901047E0FAA3E0D282
:101FDB0083F5A0C280D280EAF5A0C280D280C283F2
:101FEB00EEF8EFF974FF281E74FF39FFE87001E972
:101FFB0070BE75088F75090178081203637CEF7A40
:10200B00007B007900121EB8740212028C0247A6E4
:10201B0074F81202CBEAFEEBFFD29675A6FF7A009C
:10202B007B007900121E64D283C29275A022C280FB
:10203B00D280D292C2837AF97BC0EFFCD2838CA080
:10204B00C280D280EEF5A0C280D280C283D2838CB4
:10205B00A0C280D280F5A0C280D280C283EA1A705F
:10206B00DBEB1B70D702236974F41202CB890BECE8
:10207B0024FFF582E43416F583E493901044F0F5D5
:10208B000875090074037808120263901042E50882
:10209B00F0A3E509F08A088B09901042E0F8A3E061
:1020AB00F9E8C333F8E933F9E824FFFEE93410FF0C
:1020BB00750A08AA08AB09A90B121E6478007920CF
:1020CB00D283C29275A022C280D280D292C2837573
:1020DB000C0E8E828F83E49358FAA3E49359FBEA98
:1020EB007001EB60059010458003901047E0FCA356
:1020FB00E0D283F5A0C280D280ECF5A0C280D28062
:10210B00C283E9C313F9E813F8150CE50C70C3EEA1
:10211B0024020E0EEF3400FFE5082401F508E50953
:10212B003400F509150AE50A70897F0502032B7443
:10213B00F11202CB890AECFEED8A0C8B0D75084F60
:10214B00750906750E56750F01F50BAA0CAB0DA98B
:10215B000A121E64D283C29275A022C280D280D290
:10216B0092C2838508828509837B087C807A08E488
:10217B00935CD283600C850BA0C280D280EEF5A05D
:10218B00800A75A074C280D28075A053C280D280A1
:10219B00C283ECC313FC1AEA70D5A31BEB70CCE51E
:1021AB00082408F508E5093400F509E50C2401F5C8
:1021BB000CE50D3400F50DE50E24FFF50EE50F349F
:1021CB00FFF50FE50E7002E50F70808004C296D20A
:1021DB00967F0802032B74F81202CB901047E4F0A1
:1021EB00A3F090104974BFF0A3741DF090104574C8
:1021FB00FFF0A3F0901047E0FAA3E0FB12201B9036
:10220B00103EE0D2E0F07C8F7D017A017B007912E9
:10221B0012236E7C8F7D017A017B00790112236E74
:10222B007C8F7D017A017B0079DF12236E7C8F7DA1
:10223B00017A017B0079EF12236E7E007F0075829D
:10224B00757583198019EEFAEFFBEA75F00AA4FA9B
:10225B00ADF075F00AEBA42DFB7902122073A3E00D
:10226B00FAEE24010EEF3400FFEAFC743F6A70D6DD
:10227B007E007F0075829D7583198019EEFAEFFB46
:10228B00EA75F00AA4FAADF075F00AEBA42DFB7910
:10229B00E1122073A3E0FAEE24010EEF3400FFEA03
:1022AB00FC743F6A70D6901A51E0F8A3E0F99010D5
:1022BB0045E8F0A3E9F07582C57583197EC87F00E8
:1022CB008012EEFAEFFB7902122073EE240AFEEF76
:1022DB003400FFA3E0FAFC743F6A70E67582CE759A
:1022EB0083197E407F018012EEFAEFFB79E1122019
:1022FB0073EE240AFEEF3400FFA3E0FAFC743F6A8E
:10230B0070E6901A53E0F8A3E0F9901045E8F0A3BB
:10231B00E9F07582CE7583197E5E7F018012EEFA2D
:10232B00EFFB79E1122073EE240AFEEF3400FFA3DA
:10233B00E0FAFC743F6A70E67582C57583197E2CD2
:10234B007F018012EEFAEFFB7902122073EE240A62
:10235B00FEEF3400FFA3E0FAFC743F6A70E67F01E6
:10236B0002032B74F61202CB890A8A088B09ECFE46
:10237B00EDFF121E6490103EE0A2E0E492E0120327
:10238B00740001FF239423C023901049E0FAA3E0CB
:10239B00D283F5A0C280D280EAF5A0C280D280C2DF
:1023AB0083EEF8EFF974FF281E74FF39FFE8700114
:1023BB00E970D6803F901049E0FAA3E0D283F5A0F4
:1023CB00C280D280EAF5A0C280D280C283AA08ABB9
:1023DB0009A90A121E64E5082401F508E509340071
:1023EB00F509EEF8EFF974FF281E74FF39FFE8705A
:1023FB0001E970C17F0302032B74F71202CB90101B
:10240B004974EFF0A3747BF07508197509007E14FD
:10241B007F00AA08AB09EEF9121E64901049E0FA8E
:10242B00A3E0D283F5A0C280D280EAF5A0C280D20D
:10243B0080C283EE2405FEEF3400FFC3EE94E0EF81
:10244B00940040CEE5082419F508E5093400F50998
:10245B00C3E508948FE509940140B3750814750919
:10246B00007E007F00EEFAEFFBA908121E649010AD
:10247B0049E0FAA3E0D283F5A0C280D280EAF5A0AE
:10248B00C280D280C283EE2405FEEF3400FFC3EE80
:10249B00948FEF940140CEE5082419F508E5093433
:1024AB0000F509C3E50894E0E509940040B39010EA
:1024BB003EE0C2E0F07CC87D007AC87B0079141244
:1024CB00236EE0D2E0F07C8F7D017A007B0079787F
:1024DB0012236E0247A674F51202CB901049E0F559
:1024EB000AA3E0F50B901049E4F0A3F0901047F02D
:1024FB00A3F090103EE0C2E0F07E127F0075082939
:10250B007C0D7D00EEFAEFFB790212236E7C0D7DC4
:10251B000074012EFAE43FFB790212236EEE240ABB
:10252B00FEEF3400FF1508E50870D5E0C2E0F07E41
:10253B00127F007508297C0D7D00EEFAEFFB79E127
:10254B0012236E7C0D7D0074012EFAE43FFB79E1C2
:10255B0012236EEE240AFEEF3400FF1508E5087017
:10256B00D5901A51E0F8A3E0F9901045E8F0A3E9F3
:10257B00F07E007F007508BE8E098015AA08AB0996
:10258B007902122073E508240AF508E5093400F5F1
:10259B0009EE2400F582EF341AF583E0FAEE2401FC
:1025AB000EEF3400FFEAFC743F6A70D0901A53E0D0
:1025BB00F8A3E0F9901045E8F0A3E9F07E007F0066
:1025CB007508227509018015AA08AB09790212203A
:1025DB0073E508240AF508E5093400F509EE240A29
:1025EB00F582EF341AF583E0FAEE24010EEF340096
:1025FB00FFEAFC743F6A70D090103CE0A2E79010A9
:10260B0045500874E0F0A37407800474FFF0A3F046
:10261B007E007F0075085A8E098015AA08AB0979D0
:10262B00E1122073E508240AF508E5093400F509E1
:10263B00EE241EF582EF341AF583E0FAEE24010E38
:10264B00EF3400FFEAFC743F6A70D0901000E0702A
:10265B0011901A51E0F8A3E0F9901045E8F0A3E9C6
:10266B00801064017005901A5380E990104574FF37
:10267B00F0A3F07E007F007508148E098015AA0860
:10268B00AB0979E1122073E508240AF508E5093452
:10269B0000F509EE2414F582EF341AF583E0FAEE17
:1026AB0024010EEF3400FFEAFC743F6A70D09010E7
:1026BB004574FFF0A3F07E007F007508148E09802F
:1026CB0015AA08AB097902122073E508240AF5084C
:1026DB00E5093400F509EE24ECF582EF3419F583A6
:1026EB00E0FAEE24010EEF3400FFEAFC743F6A704F
:1026FB00D07E007F0075085A8E098015AA08AB0999
:10270B007902122073E508240AF508E5093400F56F
:10271B0009EE24F6F582EF3419F583E0FAEE240185
:10272B000EEF3400FFEAFC743F6A70D07E007F002E
:10273B007508968E098015AA08AB0979E1122073EA
:10274B00E508240AF508E5093400F509EE2428F517
:10275B0082EF341AF583E0FAEE24010EEF3400FF1A
:10276B00EAFC743F6A70D07E007F007508E68E0924
:10277B008015AA08AB0979E1122073E508240AF544
:10278B0008E5093400F509EE2432F582EF341AF529
:10279B0083E0FAEE24010EEF3400FFEAFC743F6A8B
:1027AB0070D0901049E50AF0A3E50BF07F0402030B
:1027BB002BC082C083740190102FF090103FE04427
:1027CB0012F079591228B89019EAE090101BF0908A
:1027DB00102FE090101CF0901030E090101DF09036
:1027EB001031E090101EF0740290102FF090103FFB
:1027FB00E04412F079591228B890102FE090101F76
:10280B00F0901030E0901020F0901031E0901021FB
:10281B00F0740890102FF090103FE04412F07959AB
:10282B001228B890102FE0901022F0901030E0900A
:10283B001023F0901031E0901024F0740E90102FB4
:10284B00F090103FE0C2E1F0D2E4F079591228B8D1
:10285B0090102FE0901025F0901030E0901026F0A3
:10286B00743790102FF090103FE0C2E1F0D2E4F0FB
:10287B0079591228B890102FE0901027F090103053
:10288B00E0901028F0740D90102FF090103FE0C2E4
:10289B00E1F0D2E4F079591228B890102FE09010A3
:1028AB0029F0901030E090102AF002293FC082C02E
:1028BB00837A007B0090103FA2A8E092E3F0C2A8BD
:1028CB00E99019EAF090103FE0D2E0F0A2E4500753
:1028DB00C2E4F0D2E28002C2E2F0D2C5E0A2E05044
:1028EB001BEAF8EBF97401280AE439FBC3E894E915
:1028FB00E994FD40ECE0C2E0F0C340E5901041E00C
:10290B00A2E25028E0A2E14023E4901030F09010B6
:10291B0031F0740190102FF090103FE0C2E2F0D232
:10292B00C5A2E040FC901041E0C2E2F090103FE005
:10293B00A2E392A8D083D08222C0E0C0D0E8C0E04E
:10294B00E9C0E0EAC0E0C082C083A2984003022A3B
:10295B00ED90103FE0A2E05016901018E0FA7401D1
:10296B002AF0EAC39415400C90103FE0C2E0F0E46B
:10297B00901018F0901011E07007901014E4F0A371
:10298B00F0C298E59990101AF0901011E0C39411D1
:10299B004003022AED90101AE0C0E0901014E024DE
:1029AB0001F8A3E03410F988828983D0E0F090100D
:1029BB0011E004F0901014E02401F0A3E03400F0D7
:1029CB00901011E064106003022AED901010E06487
:1029DB000D6003022AD590103CC082901001E0A23A
:1029EB00E0758310D082E092E3F090103CC08290AF
:1029FB001002E0A2E0758310D082E092E1F090101B
:102A0B003CC082901003E0A2E0758310D082E0926C
:102A1B00E2F090103CE0A2E1400DE0A2E240089011
:102A2B001004E0901036F0901005E0901030F0900C
:102A3B001006E0901031F0901007E090102FF090FE
:102A4B001008E09019EAF0901009E09019EBF09063
:102A5B00100AE0901019F090103CC08290100BE01F
:102A6B00A2E0758310D082E092E6F0901019E0643A
:102A7B00017004C2B08002D2B090103CE0A2E3E03F
:102A8B005014E0C296901034E4F0A3F0D29690105C
:102A9B003CE0C2E0800CA2E140F7E0A2E240F2E0B1
:102AAB00D2E0F090102FE06401700890103FE0D25C
:102ABB00E18010E0640260F3E0640860EE90103F88
:102ACB00E0C2E1F0E49010118017E4901011F09047
:102ADB00103CE0D2E0F0E0C2E3F0E0C2E1F0E0C293
:102AEB00E2F0A2995056C2999019E8E07002A3E067
:102AFB00603A9019E8E0F8A3E0F9901012E06870E2
:102B0B0003A3E0697007901016E4F0A3F090101A7D
:102B1B00E0F599901016E02401F0A3E03400F0905A
:102B2B0019E8E024FFF0A3E034FF800F901012E0CF
:102B3B00F8A3E0F99019E8E8F0A3E9F0D083D0828C
:102B4B00D0E0FAD0E0F9D0E0F88004D083D082D086
:102B5B00D0D0E032C0E0C0D0C082C083C0F0A2C2EF
:102B6B005003022C8074F055C01203F00003804513
:102B7B002CC0A12BE0842B802C9019EAE0C333F5F9
:102B8B00C253C2FE90103FE0A2E4E492E045C2F5CE
:102B9B00C2C2C5022C80A2C14003022C3490103F4C
:102BAB00E0A2E45003022C80901032E06401702309
:102BBB009019EAE0645D600AE064486005E06449EE
:102BCB00704290103FE0C2E0F0E4901032F0D2C4BB
:102BDB00022C8090103FE0A2E14008901032E0649C
:102BEB000260DF901032E01203740003802C012C82
:102BFB000F2C292CCD2B901032E004F090102FE0ED
:102C0B00F5C2807190103FE0A2E25007D2E4F0D2FF
:102C1B00C58062901032E004F090103080E190108B
:102C2B0032E004F090103180D6E4901032F0D2C430
:102C3B009019EAE0645D603D80D5901032E012039C
:102C4B00740101802C542C6C2CE5C2901030F09048
:102C5B001032E004F090103FE0A2E1500AD2C180A4
:102C6B0014E5C2901031F0C2C1E4901032F0901014
:102C7B003FE0C2E0F0C2C0D0F0022B56C0E0C0D0A3
:102C8B00C082C083D29090103CE0D2E4F0022B566D
:102C9B00C0E0C0D0EAC0E0C082C083901A57E0FA0F
:102CAB0074012AF0EAC39405405C75A60075A0FF79
:102CBB00C296C283901040A2A5E092E0F0A2A0E0E1
:102CCB0092E1F0A2A6E092E2F0A2A7E092E3F0A2DA
:102CDB00A2E092E4F0A2A1E092E5F0A2A3E092E6DA
:102CEB00F0A2A4E092E7F0E064FF6013901041E0E3
:102CFB00A2E4400BE0D2E3F090103CE0C2E3F0D250
:102D0B0096E4901A57F0C2CFD083D082D0E0FA026B
:102D1B002B5AC2AD901041E0D2E4F074FF901040FA
:102D2B00F07402901000F090103DE0D2E0F0E0D291
:102D3B00E1F0D2B01219DB7418901030F07440909F
:102D4B001031F0740290102FF0901041E0D2E2F0AD
:102D5B0090103FE0C2E4F0D2E1F0901041E0C2E10C
:102D6B00F079591228B8E0D2E2F0E4901033F090E9
:102D7B00103FE054EDF0901033E090102FF0795DA0
:102D8B001228B890103FE054EDF0740890102FF01B
:102D9B0079481228B890103FE054EDF07408901069
:102DAB002FF079491228B8121A7775A6FF7A537B40
:102DBB007412201B9010457437F0A374FFF0901021
:102DCB00477453F0A37474F07C377DFF7A237B0038
:102DDB00795A12213A75824F7583197E1E7F0080B6
:102DEB0012EEFAEFFB7919122073EE240AFEEF3480
:102DFB0000FFA3E0FAFC743F6A70E6D2AD9010407E
:102E0B00E064FF60F8901041E0C2E4F0C2AD122123
:102E1B00E112240490103CE0D2E5F0E0D2E3800E06
:102E2B00C296D29612304CE0C2E3F0E0D2E0F0E072
:102E3B00A2E54057E0A2E040FBE0A2E340E2E0A2C3
:102E4B00E1501F1227BC9019E87414F0A3E4F09022
:102E5B0010127414F0A3E4F0D29990103CE0C2E18C
:102E6B0080C8E0A2E250C890103FE0C2E4F0901995
:102E7B00EAE0F91228B87401901A50F090103CE077
:102E8B00C2E280A61227BCE0C2E1F090103CE0A2A7
:102E9B00E5400302304B800AE0A2E15005C2AD12BF
:102EAB0036D3D2AD90103CE0A2E3E0502FA2E75016
:102EBB0007C2AD123B7A80EA90103DE0FAE0FBEAE4
:102ECB00A2E0500CEBA2E15007C2AD12385880D2F1
:102EDB00E0A2E050C3C2AD12354C80C6A2E140A4C3
:102EEB00E0A2E2502190103FE0C2E4F09019EAE03A
:102EFB00F91228B87401901A50F090103CE0C2E21D
:102F0B00F0E0D2E38084901041E0A2E34003022E74
:102F1B009690103CE0C2E2F0901040E0A2E2407FBD
:102F2B00901033E06410F090103FE054EDF09010EF
:102F3B0033E090102FF0795D1228B8901A51E0F819
:102F4B00A3E0F9901045E8F0A3E9F0901033E0A26C
:102F5B00E440267582CE7583197E407F01E0FAFC32
:102F6B00743F6A603AEEFAEFFB79E1122073EE24BC
:102F7B000AFEEF3400FFA380E47582D27583197EBD
:102F8B00407F018012EEFAEFFB79E1122073EE2401
:102F9B000AFEEF3400FFA3E0FAFC743F6A70E69080
:102FAB001040E0A2E3407F901033E06420F09010DB
:102FBB003FE054EDF0901033E090102FF0795D125C
:102FCB0028B8901A53E0F8A3E0F9901045E8F0A365
:102FDB00E9F0901033E0A2E540267582CE75831997
:102FEB007E5E7F01E0FAFC743F6A603AEEFAEFFB1B
:102FFB0079E1122073EE240AFEEF3400FFA380E484
:10300B007582D27583197E5E7F018012EEFAEFFB1B
:10301B0079E1122073EE240AFEEF3400FFA3E0FAED
:10302B00FC743F6A70E6C2AD123D2B901041E0C2BA
:10303B00E3F090103CE0A2E25003022E96022F0C1C
:10304B0022C082C083D2A8C29090103CE0A2E45070
:10305B00F8E0C2E4F0C2A8D290901036E0600464AD
:10306B00027033901034E4F0A3F0D297C297D2974A
:10307B00901034E02401F0A3E03400F0901034C33E
:10308B00E094FFA3E0940140E1D297901012E4F09A
:10309B00A37402F0D299901019E064016005E0640A
:1030AB0002700890103CE0A2E650F8901036E064F5
:1030BB00016005E064027031901034E4F0A3F0D2AB
:1030CB0095C295D295901034E02401F0A3E0340022
:1030DB00F0901034C3E094FFA3E0940140E1901012
:1030EB0012E4F0A37402F0D299C296D29602293F51
:1030FB0074F51202CB7E00E4901947F075A60075AB
:10310B00A0FF786B79137A10C297E5A0244FF58254
:10311B00E43404F583E49388828983F0A3E4F0D24A
:10312B0097E824020808E93400F91AEA70DA7F08F4
:10313B00787B7913C297E82410FAE93400FBE5A0F9
:10314B00244FF582E43404F583E4938A828B83F075
:10315B00A3E4F0D297EE705B901A58E0F5088882E2
:10316B008983E0FCA3E0FD74FC2508F50A74FF34A9
:10317B0000F50BC3E50A9CE50B9DA2D265D033503D
:10318B003274042508F508E43400F509EC9508EDD4
:10319B009509A2D265D033501A8A828B83E0FAC389
:1031AB00EC9AED9400A2D265D0335007EF901947FB
:1031BB00F07E010FE824020808E93400F9EFC3940C
:1031CB005C500302313F0227B774F41202CB750A2D
:1031DB0000E4901947F075A60075A0FF7853791796
:1031EB007A10C295E5A0244FF582E43404F583E40C
:1031FB009388828983F0D295A3A882A9831AEA7057
:10320B00E1750B08785B7917C295E82408FAE93465
:10321B0000FBE5A0244FF582E43404F583E4938AA4
:10322B00828B83F0D295E50A704E88828983E0F514
:10323B0082AE82901A58E0FC74FC2CF50874FF34B3
:10324B0000F509C3E5089EE5099400A2D265D033C9
:10325B00502674042CFCE43400FDEE9CE49DC36505
:10326B00D03350148A828B83E0FAEEC39A5009E56F
:10327B000B901947F0750A01050B88828983A3A867
:10328B0082A983E50BC3945C5003023213022135F0
:10329B0074F21202CB7E00E4901947F075A600750C
:1032AB00A0FF7A537B17786B79137C10C297E5A03C
:1032BB00244FF582E43405F583E493F5088882897D
:1032CB0083F0A3E4F0D297C295E5A0244FF582E4F6
:1032DB003405F583E4938A828B83F0D295E824023C
:1032EB000808E93400F9A3AA82AB831CEC70BD7FFC
:1032FB00087C5B7D177A7B7B13C297EA2410F8EB73
:10330B003400F9880A890BE5A0244FF582E43405D3
:10331B00F583E49388828983F0A3E4F0D297C29576
:10332B00EC2408F8ED3400F9880C890DE5A0244F46
:10333B00F582E43405F583E49388828983F0D29592
:10334B00EE600302340D901000E07065901A58E0A7
:10335B00F88A828B83E0F508A3E0F50974FC28F565
:10336B000C74FF3400F50DC3E50C9508E50D9509BC
:10337B00A2D265D033400302340D740428F8E43430
:10338B0000F9E50898E50999A2D265D03350738509
:10339B000A82850B83E0F8A3E0F9C3E50898E509F9
:1033AB0099A2D265D033505AEF901947F07E018025
:1033BB00516401704D8C828D83E0F50EF582858210
:1033CB0008901A58E0F874FC28F50A74FF3400F5DD
:1033DB000BC3E50A9508E50B9400A2D265D03350D8
:1033EB0021740428F8E43400F9E50898E499C365DE
:1033FB00D033500E850C82850D83E0F8E50EC39813
:10340B0040A60FEA24020A0AEB3400FB8C828D8360
:10341B00A3AC82AD83EFC3945C50030233047F07EC
:10342B0002032B74F51202CB7E00E4901947F07562
:10343B00A60075A0FF786B79137A08C297E5A024D4
:10344B004FF582E43404F583E49388828983F0A3F7
:10345B00E4F0D297C295E5A0244FF582E43404F54D
:10346B0083E49388828983A3A3F0A3E4F0D295E845
:10347B002404F8E93400F91AEA70C07F08787B79E4
:10348B0013C297E82410FAE93400FBE5A0244FF5AA
:10349B0082E43404F583E4938A828B83F0A3E4F013
:1034AB00D297C295E5A0244FF582E43404F583E46A
:1034BB0093FCE82412F582E93400F583ECF0A3E4E5
:1034CB00F0D295EE7065901000E06402605D901A8A
:1034DB0058E0F50888828983E0FCA3E0FD74FC25A5
:1034EB0008F50A74FF3400F50BC3E50A9CE50B9D48
:1034FB00A2D265D033503474042508F508E43400A7
:10350B00F509EC9508ED9509A2D265D033501C8ACC
:10351B00828B83E0FAA3E0FBC3EC9AED9BA2D2650E
:10352B00D0335007EF901947F07E010F0FE82404BA
:10353B00F8E93400F9EFC3945B500302348C022793
:10354B00B774F11202CBD2A8C29090103CE0A2E467
:10355B0050F8E0C2E4F0C2A81230FB901000E06417
:10356B000270087401901947F08009901947E070B8
:10357B00030236D07E007F0075084B750910750E5F
:10358B0033750F14E0C333F8E433F9E8246BF50C0F
:10359B00E93413F50D75A60075A0FFC297E5A024BD
:1035AB004FF582E43404F583E493850E82850F8313
:1035BB00F0A3E4F0D29775A6FF850882850983E016
:1035CB00FC74786C600874C86E7001EF700B90100F
:1035DB004974EFF0A3747B8052EC75F00584E5F031
:1035EB007011EEF8EFF97A197B001201FAEA70010B
:1035FB00EB60DB8C0A7405250AF8E43400F97A19C0
:10360B007B001201F2EA7001EB7011EEF8EFF97A20
:10361B00057B001201FAEA7001EB60B2901047E0F3
:10362B00F8A3E0F9901049E8F0A3E9F0EEFAEFFB0C
:10363B00ECF9121E64901049E0FAA3E0D283F5A0D6
:10364B00C280D280EAF5A0C280D280C283901A5188
:10365B00E0F8A3E0F9901049E8F0A3E9F0850C82BB
:10366B00850D83E024F8F50AEEFAEFFBA90A121E8A
:10367B0064901049E0FAA3E0D283F5A0C280D28017
:10368B00EAF5A0C280D280C283850882850983E5D2
:10369B000AF0EE24010EEF3400FFE50C2402F50CCA
:1036AB00E50D3400F50DE50E2402F50EE50F3400A3
:1036BB00F50FA3858208858309C3EE948FEF9401E0
:1036CB0050030235A00221D874F11202CBD2A8C24A
:1036DB009090103CE0A2E450F8E0C2E4F0C2A812D3
:1036EB0031D4901000E0640270087401901947F017
:1036FB008009901947E070030238557E007F0075F2
:10370B000EB7750F177508DB750911E02453F50C0F
:10371B00E43417F50D75A60075A0FFC295E5A0243E
:10372B004FF582E43404F583E493850E82850F8391
:10373B00F0D29575A6FF850882850983E0FC747825
:10374B006C600874C86E7001EF700B90104974EFC9
:10375B00F0A3747B8052EC75F00584E5F07011EEEC
:10376B00F8EFF97A197B001201FAEA7001EB60DBD2
:10377B008C0A7405250AF8E43400F97A197B0012D7
:10378B0001F2EA7001EB7011EEF8EFF97A057B00AC
:10379B001201FAEA7001EB60B2901047E0F8A3E077
:1037AB00F9901049E8F0A3E9F0EEFAEFFBECF9120F
:1037BB001E64901049E0FAA3E0D283F5A0C280D238
:1037CB0080EAF5A0C280D280C283901A53E0F8A39E
:1037DB00E0F9901049E8F0A3E9F0850C82850D83A0
:1037EB00E024F8F50AEEFAEFFBA90A121E6490101A
:1037FB0049E0FAA3E0D283F5A0C280D280EAF5A01B
:10380B00C280D280C283850882850983E50AF0EEE7
:10381B0024010EEF3400FF850C82850D83A3858276
:10382B000C85830D850882850983A3858208858392
:10383B0009850E82850F83A385820E85830FC3EEC8
:10384B00948FEF940150030237200221D874F112A8
:10385B0002CB74FA120276D2A8C29090103CE0A26E
:10386B00E450F8E0C2E4F0C2A812329B901000E0E2
:10387B00640270087401901947F08009901947E0B1
:10388B007003023B6E7E007F0074041202C174B79A
:10389B00F0A37417F0750C4B750D107508DB7509DB
:1038AB0011901947E0F82453FAE43417FB74021211
:1038BB0002C1EAF0A3EBF08510828511837433F01B
:1038CB00A37414F0E8C333F8E433F9E8246BF50E72
:1038DB00E93413F50F75A60075A0FFC297E5A02478
:1038EB004FF582E43405F583E493FA851082851154
:1038FB0083E0F8A3E0F5838882EAF0A3E4F0D297A3
:10390B00C295E5A0244FF582E43405F583E493C01A
:10391B00E074041202C1E0F8A3E0F5838882D0E0E2
:10392B00F0D29575A6FF850C82850D83E0FC74782B
:10393B006C600874C86E7001EF700B90104974EFD7
:10394B00F0A3747B8052EC75F00584E5F07011EEFA
:10395B00F8EFF97A197B001201FAEA7001EB60DBE0
:10396B008C0A7405250AF8E43400F97A197B0012E5
:10397B0001F2EA7001EB7011EEF8EFF97A057B00BA
:10398B001201FAEA7001EB60B2901047E0F8A3E085
:10399B00F9901049E8F0A3E9F0EEFAEFFBECF9121D
:1039AB001E64901049E0FAA3E0D283F5A0C280D246
:1039BB0080EAF5A0C280D280C28385088285098304
:1039CB00E0FC74786C600874C86E7001EF700B903B
:1039DB00104974EFF0A3747B8052EC75F00584E50D
:1039EB00F07011EEF8EFF97A197B001201FAEA7018
:1039FB0001EB60DB8C0A7405250AF8E43400F97AD4
:103A0B00197B001201F2EA7001EB7011EEF8EFF97D
:103A1B007A057B001201FAEA7001EB60B290104755
:103A2B00E0F8A3E0F9901049E8F0A3E9F0EEFAEF23
:103A3B00FBECF9121E64901049E0FAA3E0D283F577
:103A4B00A0C280D280EAF5A0C280D280C283901A35
:103A5B0051E0F8A3E0F9901049E8F0A3E9F0850EE6
:103A6B0082850F83E0246AF50AEEFAEFFBA90A12AE
:103A7B001E64901049E0FAA3E0D283F5A0C280D275
:103A8B0080EAF5A0C280D280C283850C82850D832B
:103A9B00E50AF0901A53E0F8A3E0F9901049E8F02A
:103AAB00A3E9F074021202C1E0F8A3E0F583888267
:103ABB00E02406F50AEEFAEFFBA90A121E64901039
:103ACB0049E0FAA3E0D283F5A0C280D280EAF5A048
:103ADB00C280D280C283850882850983E50AF0EE15
:103AEB0024010EEF3400FFE50E2402F50EE50F3432
:103AFB0000F50F851082851183E02402F8A3E034D2
:103B0B0000F9851082851183E8F0A3E9F0740212A5
:103B1B0002C1E02401F8A3E03400F974021202C1DF
:103B2B00E8F0A3E9F0850882850983A385820885DF
:103B3B008309850C82850D83A385820C85830D7487
:103B4B00041202C1E02401F8A3E03400F97404125A
:103B5B0002C1E8F0A3E9F0C3EE948FEF9401500398
:103B6B000238E0C296D296740612028C0221DC74E3
:103B7B00F31202CBD2A8C29090103CE0A2E450F812
:103B8B00E0C2E4F0C2A812342E901000E064027080
:103B9B00087401901947F08009901947E0700302EF
:103BAB003D2275A60075A0FF7E007F007833791447
:103BBB00C297E5A0244FF582E43404F583E493889F
:103BCB00828983F0A3E4F0D297C295E5A0244FF548
:103BDB0082E43404F583E49388828983A3A3F0A35E
:103BEB00E4F0D295EE24020E0EEF3400FFE824042D
:103BFB00F8E93400F9C3EE948EEF940140B275A648
:103C0B00FF7E007F0075084B750910901947E0C3C4
:103C1B0033F8E433F9E8246BF50CE93413F50D852F
:103C2B000882850983E0FC74786C600874C86E7038
:103C3B0001EF700B90104974EFF0A3747B8052EC82
:103C4B0075F00584E5F07011EEF8EFF97A197B0049
:103C5B001201FAEA7001EB60DB8C0A7405250AF895
:103C6B00E43400F97A197B001201F2EA7001EB706F
:103C7B0011EEF8EFF97A057B001201FAEA7001EB0D
:103C8B0060B2901047E0F8A3E0F9901049E8F0A378
:103C9B00E9F0EEFAEFFBECF9121E64901049E0FA32
:103CAB00A3E0D283F5A0C280D280EAF5A0C280D275
:103CBB0080C28390104974FFF0A3F0850C82850DB0
:103CCB0083E024F8F50AEEFAEFFBA90A121E6490C2
:103CDB001049E0FAA3E0D283F5A0C280D280EAF5C6
:103CEB00A0C280D280C283850882850983E50AF051
:103CFB00EE24010EEF3400FFE50C2402F50CE50D6C
:103D0B003400F50DA3858208858309C3EE948FEFEC
:103D1B0094015003023C2AC296D2967F0602032BD3
:103D2B0074F41202CB901049E0F50AA3E0F50B9066
:103D3B001049E4F0A374F8F0901040E0A2E7E4928D
:103D4B00E044FEF4FA901037E02AF0901040E0A225
:103D5B00E6E492E044FEF4FA901037E0C39AF06484
:103D6B00FF700474088007E0C394094002E4F090EC
:103D7B00194EE0FA901037E06A60031224E1901AB2
:103D8B0055E0F8A3E0F9901047E8F0A3E9F09010A4
:103D9B004574FFF0A3F0901037E012037400083263
:103DAB0044BE3DC43D3B3EBC3E483FD23F4C4034FD
:103DBB0043B24312444E02443290103EE0C2E0F054
:103DCB007E127F007508077C0D7D00EEFAEFFB7904
:103DDB000212236E7C0D7D0074012EFAE43FFB79F9
:103DEB000212236EEE240AFEEF3400FF1508E508DD
:103DFB0070D57E007F007508148E09EE24ECF582D9
:103E0B00EF3419F583E0FAEE24010EEF3400FFEAEC
:103E1B00FC743F6A700302432AAA08AB09790212A9
:103E2B002073E508240AF508E5093400F50980CB71
:103E3B0090103EE0C2E0F07E587F0075080A7C0DC2
:103E4B007D00EEFAEFFB790212236E7C0D7D007480
:103E5B00012EFAE43FFB790212236EEE240AFEEFE9
:103E6B003400FF1508E50870D57E007F0075085AF1
:103E7B008E098015AA08AB097902122073E5082474
:103E8B000AF508E5093400F509EE24F6F582EF345E
:103E9B0019F583E0FAEE24010EEF3400FFEAFC740F
:103EAB003F6A70D0901047E4F0A3F012453C0244F7
:103EBB003290103EE0C2E0F07EBC7F0075080A7CB9
:103ECB000D7D00EEFAEFFB790212236E7C0D7D0067
:103EDB0074012EFAE43FFB790212236EEE240AFEE4
:103EEB00EF3400FF1508E50870D5901A51E0F8A3E0
:103EFB00E0F9901045E8F0A3E9F07E007F0075082B
:103F0B00BE8E098015AA08AB097902122073E50849
:103F1B00240AF508E5093400F509EE2400F582EFD3
:103F2B00341AF583E0FAEE24010EEF3400FFEAFCBD
:103F3B00743F6A70D079001248F002443290103E00
:103F4B00E0C2E0F07E207F0175080A7C0D7D00EE5B
:103F5B00FAEFFB790212236E7C0D7D0074012EFAB1
:103F6B00E43FFB790212236EEE240AFEEF3400FFCE
:103F7B001508E50870D5901A53E0F8A3E0F99010F6
:103F8B0045E8F0A3E9F07E007F0075082275090172
:103F9B008015AA08AB097902122073E508240AF5EB
:103FAB0008E5093400F509EE240AF582EF341AF519
:103FBB0083E0FAEE24010EEF3400FFEAFC743F6A53
:103FCB0070D07901023F4290103EE0C2E0F07E12C9
:103FDB007F007508077C0D7D00EEFAEFFB79E1128F
:103FEB00236E7C0D7D0074012EFAE43FFB79E11208
:103FFB00236EEE240AFEEF3400FF1508E50870D59A
:10400B007E007F007508148E098015AA08AB09790C
:10401B00E1122073E508240AF508E5093400F509D7
:10402B00EE2414F582EF341AF583E0FAEE24010E38
:10403B00EF3400FFEAFC743F6A70D01247AB0244C6
:10404B003290103EE0C2E0F07E587F007508067C8F
:10405B000D7D00EEFAEFFB79E112236E7C0D7D00F6
:10406B0074012EFAE43FFB79E112236EEE240AFE73
:10407B00EF3400FF1508E50870D57E007F0075084A
:10408B005A8E098015AA08AB0979E1122073E5084D
:10409B00240AF508E5093400F509EE241EF582EF34
:1040AB00341AF583E0FAEE24010EEF3400FFEAFC3C
:1040BB00743F6A70D090103CE0A2E740030241A924
:1040CB00901040E0A2E5500302428C90103CE0C2FD
:1040DB00E7F0901047E4F0A3F075088F75090178AD
:1040EB00081203637CDE7A007B007914121F87743D
:1040FB000212028C1224047E487F1990103AE0F8C9
:10410B00A3E0F9E875F006A4F8AAF075F006E9A4A7
:10411B002AF9E8246FFAE93418FBEAF8EBF97CEC9E
:10412B007D1975080588828983E493F5098E828F42
:10413B0083F0EC240BF582ED3400F583E509F08C6C
:10414B00828D83A3AC82AD8388828983A3A882A945
:10415B00838E828F83A3AE82AF831508E50870C56B
:10416B008A828B83A3A3A3A3A3E49390194DF0900E
:10417B001047E4F0A3F07582487583197E64FFE065
:10418B00FAFC743F6A700302428CEEFAEFFB790281
:10419B00122073EE240AFEEF3400FFA380E1E0A2AD
:1041AB00E7500302428C901040E0A2E4500302421D
:1041BB008C90103CE0D2E7F0901047E4F0A3F07540
:1041CB00088F75090178081203637CDE7A007B0087
:1041DB007914121F87740212028C1224047E487FFA
:1041EB001990103AE0F8A3E0F9E875F006A4F8AAE4
:1041FB00F075F006E9A42AF9E82417FAE93419FB5B
:10420B00EAF8EBF97CEC7D1975080588828983E463
:10421B0093F5098E828F83F0EC240BF582ED34003D
:10422B00F583E509F08C828D83A3AC82AD83888204
:10423B008983A3A882A9838E828F83A3AE82AF8347
:10424B001508E50870C58A828B83A3A3A3A3A3E4F7
:10425B009390194DF0901047E4F0A3F075824875D8
:10426B0083197E64FF8012EEFAEFFB790212207342
:10427B00EE240AFEEF3400FFA3E0FAFC743F6A70F1
:10428B00E6901047E4F0A374F8F090103CE0A2E73E
:10429B005038C2B07480901A58F090104574E0F00A
:1042AB00A37407F07582D67583197E647F00E0FADC
:1042BB00FC743F6A6069EEFAEFFB79E1122073EE52
:1042CB00240AFEEF3400FFA380E490103DE0FAE0F7
:1042DB00FBEAA2E05009EBA2E150047440800CE031
:1042EB00A2E04005E0A2E150067480901A58F0D28B
:1042FB00B090104574FFF0A3F07582D67583197ECC
:10430B00647F008012EEFAEFFB79E1122073EE244A
:10431B000AFEEF3400FFA3E0FAFC743F6A70E690EC
:10432B001047E4F0A3F002443290103EE0C2E0F0FC
:10433B007E947F007508087C0D7D00EEFAEFFB790B
:10434B00E112236E7C0D7D0074012EFAE43FFB79A4
:10435B00E112236EEE240AFEEF3400FF1508E50888
:10436B0070D57E007F007508968E098015AA08AB64
:10437B000979E1122073E508240AF508E5093400F0
:10438B00F509EE2428F582EF341AF583E0FAEE24D2
:10439B00010EEF3400FFEAFC743F6A70D0901047B7
:1043AB00E4F0A3F0F9807D90103EE0C2E0F07EE4F3
:1043BB007F007508087C0D7D00EEFAEFFB79E112AA
:1043CB00236E7C0D7D0074012EFAE43FFB79E11224
:1043DB00236EEE240AFEEF3400FF1508E50870D5B6
:1043EB007E007F007508E68E098015AA08AB097957
:1043FB00E1122073E508240AF508E5093400F509F4
:10440B00EE2432F582EF341AF583E0FAEE24010E36
:10441B00EF3400FFEAFC743F6A70D0901047E4F071
:10442B00A3F0790112486C901047E4F0A3F09010C0
:10443B0049E50AF0A3E50BF0901037E090194EF028
:10444B0002213574F71202CB90103CE0A2E7500327
:10445B00024539901040E0A2E05005E0A2E1402572
:10446B00901047E4F0A3F075088F750901780812D6
:10447B0003637CDE7A007B007914121F87740212AF
:10448B00028C12240490103DE0FAE0FBEAA2E0500B
:10449B0025EBA2E15020901040E0A2E040079010E5
:1044AB003DE0C2E0F0901040E0A2E1405C90103D96
:1044BB00E0C2E1F08053E0A2E0501F901040E0A278
:1044CB00E0400790103DE0C2E0F0901040E0A2E128
:1044DB00403790103DE0D2E180D9E0A2E19010404E
:1044EB00E05015A2E0400790103DE0D2E0F09010B4
:1044FB0040E0A2E1401380B5A2E0400890103DE0FF
:10450B00D2E080AFE0A2E150C990103DE0FAE0FBB1
:10451B00EAA2E05009EBA2E150047440800CE0A247
:10452B00E04005E0A2E150067480901A58F0024773
:10453B00A674F71202CB90104574FFF0A3F0901005
:10454B0040E0A2E450030245DD901041E0A2E09070
:10455B00103A5025E02401F0A3E03400F090103A1B
:10456B00C3E0941CA3E09400A2D265D033403C90EE
:10457B00103A741BF0A3E48031C3E09418A3E094C9
:10458B0000A2D265D03390103AE040102401F0A382
:10459B00E03400F0901041E0D2E0800E2401F0A353
:1045AB00E03400F0901041E0C2E0F0901041E0C226
:1045BB00E1F0E0A2E150547418901038F074409080
:1045CB001039F0740290102FF0901041E0D2E202FB
:1045DB0046B8E0A2E5402B90103AE024FFF0F8A398
:1045EB00E034FFF0F9C3E89401E99400A2D265D05E
:1045FB003350B890103AE4F0A3F0901041E0D2E1C0
:10460B0080AF901047E4F0A30247A5E0A2E0504C26
:10461B0090103AE0F508A3E0F50978081203AA1800
:10462B000003634637464A464E4657467418901069
:10463B0038F0E4901039F0901041E0C2E08018742B
:10464B0018800B7419901038F0E4800874199010CE
:10465B0038F07480901039F07402804EE0A2E25072
:10466B0004741880E090103AE0F8A3E0F9E8C33343
:10467B00F8E933F9E82437F582E93418F583E49344
:10468B00C0E0740193F583D082AA82AB838A088B36
:10469B000974027808120253E508901038F0EAC446
:1046AB00333354C0901039F0740190102FF075080B
:1046BB00007E487F1990103AE0F8A3E0F9E875F016
:1046CB0006A4F8AAF075F006E9A42AF9E82417FA6B
:1046DB00E93419FBE8246FF8E93418F97CEC7D19FF
:1046EB0090103CE0A2E750068A828B83800488827C
:1046FB008983E4938E828F83F0E508C39405501071
:10470B00E0C0E0EC240BF582ED3400F583D0E0F053
:10471B0005088C828D83A3AC82AD8388828983A3A9
:10472B00A882A9838A828B83A3AA82AB838E828F72
:10473B0083A3AE82AF83E508C3940640A3901047D2
:10474B00E4F0A374F8F07582487583197E647F00DA
:10475B008012EEFAEFFB7902122073EE240AFEEFC1
:10476B003400FFA3E0FAFC743F6A70E6901047E454
:10477B00F0A3F0901038E0901030F0901039E090EA
:10478B001031F090103CE0C2E3F0E0D2E2F0901078
:10479B003FE0D2E1F074599019EAF07F0202032B4B
:1047AB0074F81202CB901040E0A2E0404D90100044
:1047BB00E06016901A51E0F8A3E0F9901045E8F08C
:1047CB00A3E9F0E4901000800A7402F09010457495
:1047DB00FFF0A3F07582DB7583197E1E7F00E0FA74
:1047EB00FC743F6A6069EEFAEFFB79E1122073EE1D
:1047FB00240AFEEF3400FFA380E4E0A2E1405090D6
:10480B001000E064016017901A53E0F8A3E0F990F0
:10481B001045E8F0A3E9F07401901000800A7402CF
:10482B00F090104574FFF0A3F07582DB7583197E51
:10483B001E7F008012EEFAEFFB79E1122073EE245B
:10484B000AFEEF3400FFA3E0FAFC743F6A70E690B7
:10485B001047E4F0A3F090104574FFF0A3F002238F
:10486B006974F71202CB901040E0A2E04055E9705A
:10487B0052901047E4F0A3F075088F750901780882
:10488B001203637CDE7A007B007914121F8774029B
:10489B0012028C90104574FFF0A3F07582E17583C2
:1048AB00197E147F008012EEFAEFFB79BE12207393
:1048BB00EE240AFEEF3400FFA3E0FAFC743F6A70AB
:1048CB00E680FEE0A2E440047A018007E0A2E54026
:1048DB00117AFFE97007EA25EAF5EA8005EA25FC7B
:1048EB00F5FC0247A674F71202CBE96003024A07F4
:1048FB00901040E0A2E4400F901A59E004F0C394EA
:10490B0008401974078014E0A2E55003024B2A906B
:10491B001A59E014F0C394C94002E4F07E007A48BF
:10492B007B1978EC79198E08901A59E075F005A46B
:10493B00240FFCE5F03418FDE5082CF582E43DF579
:10494B0083E4938A828B83F0C0E0E82415F582E937
:10495B003400F583D0E0F00E88828983A3A882A966
:10496B00838A828B83A3AA82AB83EEC3940440B663
:10497B00901A59E075F005A42413F582E5F034186C
:10498B00F583E49390194CF07582487583197EC8B2
:10499B007F008012EEFAEFFB7902122073EE240AED
:1049AB00FEEF3400FFA3E0FAFC743F6A70E6901A46
:1049BB0059E0C39405901033E04004C2E08002D26A
:1049CB00E0F090103FE054EDF0901033E090102F9A
:1049DB00F0795D1228B890103FE054EDF0901A5921
:1049EB00E0C333F8E433F9E824FFF582E93417F533
:1049FB0083E49390102FF07948024B18740169608F
:104A0B0003024B1B901040E0A2E4400F901A5AE0B7
:104A1B0004F0C39408401974078014E0A2E5500316
:104A2B00024B2A901A5AE014F0C394C94002E4F0E6
:104A3B007E007A487B1978EC79198E08901A5AE027
:104A4B0075F005A4240FFCE5F03418FDE5082CF5F2
:104A5B0082E43DF583E4938A828B83F0C0E0E82403
:104A6B001FF582E93400F583D0E0F00E888289834C
:104A7B00A3A882A9838A828B83A3AA82AB83EEC36A
:104A8B00940440B6901A5AE075F005A42413F582ED
:104A9B00E5F03418F583E49390194CF07582487562
:104AAB0083197E2C7F018012EEFAEFFB7902122024
:104ABB0073EE240AFEEF3400FFA3E0FAFC743F6AA6
:104ACB0070E6901A5AE0C39405901033E04004C28C
:104ADB00E18002D2E1F090103FE054EDF090103302
:104AEB00E090102FF0795D1228B890103FE054ED54
:104AFB00F0901A5AE0C333F8E433F9E824FFF58257
:104B0B00E93417F583E49390102FF079491228B804
:104B1B00901047E4F0A3F090104574FFF0A3F0025F
:024B2B0047A69B
:040000050000009166
:00000001FF
